:020000040000FA
:06080000F5EF22F01200EA
:06080800BBEF05F0120039
:0608180022EF04F01200C3
:06082A0002002D46000053
:10083000D20100000200000029460000CC010000A7
:0408400004000000B0
:0C084400D8CFE4FFE0CFE4FFE46EDACF91
:10085000E4FFE2CFDAFFE9CFE4FFEACFE4FFF3CF32
:10086000E4FFF4CFE4FFE6529EA201D19E92030E74
:10087000386E0E50EA6A510FE96E010EEA22EF500F
:10088000385C30E10E50E96EEA6AD890E936EA3613
:10089000690EE926010EEA22EECF38F0EFCF39F0EB
:1008A00039C038F0396A3850D76E0E50E96EEA6AAE
:1008B000D890E936EA36690EE926010EEA22EECF33
:1008C00038F0EFCF39F03850D66EF28AF294D58EE8
:1008D0000E50EA6A510FE96E010EEA22040EEF6E25
:1008E0000E50106E020E386E0F50EA6A510FE96E0C
:1008F000010EEA22EF50385C49E10F50E96EEA6AD6
:10090000D890E936EA36690EE926010EEA22EE5061
:10091000ED1009E10F50EA6A510FE96E010EEA226B
:10092000010EEF6E33D0080E0F5C0CE2070E0F14B1
:10093000386E010E385204E0E846FE0B3806FCE142
:1009400089121AD0100E0F5C0CE2070E0F14386ECD
:10095000010E385204E0E846FE0B3806FCE18A122C
:100960000BD0070E0F14386E010E385204E0E84623
:10097000FE0B3806FCE18B120F50EA6A510FE96E4C
:10098000010EEA22030EEF6E0F500E6E0F2A060EB6
:100990000F5C03E1080E0F6E0AD0130E0F5C03E12B
:1009A000160E0F6E04D0180E0F5C01E10F6A000ED8
:1009B000D8800254000E03542EE2112A000E122297
:1009C0000250115C0350125826E3116A126A030E9A
:1009D000065C1FE20450EA6A480FE96E010EEA2243
:1009E00080CFEFFF0450EA6A4B0FE96E010EEA2256
:1009F00081CFEFFF0450EA6A4E0FE96E010EEA2242
:100A000082CFEFFF042A030E045C01E3046A062A86
:100A100002D0026A036A000ED8800754000E085400
:100A200019E20C50000816E2132A000E1422075097
:100A3000135C085014580EE3136A146A030E0B5C1F
:100A400007E2092A030E095C01E3096A0B2A02D0B6
:100A5000076A086A0C5000080AE2156A1550040D6E
:100A6000F328C26E9E9C9F9C9D8CC280C2829EACCD
:100A70002DD09E9CC4503C6E3CC03DF03C6AC3509F
:100A800000013C103A6E3DC03BF01550060DF3CF0F
:100A900038F0F4CF39F0000E3826010E3922095013
:100AA000020D3850F324E96E3950F420EA6E3AC052
:100AB000EEFF3BC0EDFF152A0C50155C02E39D9C38
:100AC00005D01550040DF328C26EC282F2A442D0A4
:100AD000D59EF294F29A040E386E1050EA6A510FC5
:100AE000E96E010EEA22EF50385C34E1080E105C2A
:100AF0000DE2070E1014386E010E385204E0E8467D
:100B0000FE0B3806FCE1E81C89161CD0100E105CA8
:100B10000DE2070E1014386E010E385204E0E8465C
:100B2000FE0B3806FCE1E81C8A160CD0070E1014E8
:100B3000386E010E385204E0E846FE0B3806FCE140
:100B4000E81C8B161050EA6A510FE96E010EEA227A
:100B5000020EEF6EE552E5CFF4FFE5CFF3FFE5CFF0
:100B6000EAFFE5CFE9FFE5CFDAFFE550E5CFE0FFAB
:100B7000E5CFD8FF1000DACFE4FFE2CFDAFFE6528C
:100B8000E552E5CFDAFF1100D9CFE6FFE1CFD9FF7B
:100B9000020EE126896A92680F0EC16EC2900C6A3D
:100BA000070EB46E8A6A93688B6A9468FC0E8B1683
:100BB000FC0E941694840101010EBE6F0101D269EE
:100BC000D3690A6A096A0B6A056A046A066A026AD4
:100BD000036A076A086A116A126A136A146A156A54
:100BE000CA82CA80CA9CCA9ACA88CA96FA0ECB6EB2
:100BF000DF6ADFCF2AF00C0EE76E2A18E8AE02D0CB
:100C0000E73402D0E7502A5C38E2010EDB6A010EBD
:100C1000DBCF2AF0030EE76E2A18E8AE02D0E734E5
:100C200002D0E7502A5C27E2DFCF2AF02B6A2ABEE7
:100C30002B68060E2B02F3CF2BF0060E2A02F3CF01
:100C40002AF0F4502B26000E2A26010E2B22010E2C
:100C5000DBCF2CF02D6A2CBE2D68D8902C362D368B
:100C60002A502C24E96E2B502D20EA6EEE6AED6A94
:100C7000010EDB2ACCD7DF2ABCD70101B86B0101FA
:100C8000B96B0101B66B0101B76B0101BA6B0101D0
:100C9000BB6B0101BC6B0101BD6B0E6A0F6A106A70
:100CA000DF6ADFCF2AF0180EE76E2A18E8AE02D00E
:100CB000E73402D0E7502A5C1BE2DFCFE9FFEA6AA3
:100CC000E9BEEA68D890E936EA36690EE926010EEF
:100CD000EA22EE6AED6ADFCFE9FFEA6AE9BEEA6876
:100CE000510EE926010EEA22010EEF6EDF2AD9D756
:100CF000D586D59AD59CF294F29AF194D08ECA9466
:100D00009D829F92F28EF28CCA84020EE15C02E216
:100D1000E16AE552E16EE552E7CFD9FF1200D9CF83
:100D2000E6FFE1CFD9FF020EE126010EDB6A0101E9
:100D3000996B19EC13F00650000809E20AEC0BF06D
:100D4000052A030E055C01E1056A0606F4D70B507F
:100D5000000809E236EC0BF00A2A030E0A5C01E1F6
:100D60000A6A0B06F4D7040104011851800B6CE1E8
:100D7000060E0101C85D68E36D50020B65E10101DB
:100D8000996B040119510101995D53E201019951D7
:100D9000EA6A080FE96E050EEA22EFCFDFFF0101D4
:100DA000CC511CE10D0E2A6EDF502A5C05E00A0EC4
:100DB0002B6EDF502B5C12E10101010ECC6F0101A3
:100DC000B851EA6A4A0FE96E020EEA220D0EEF6E82
:100DD0000101B82BDE52010EDD6E15D00D0EDF5C69
:100DE00011E00A0EDF5C0EE00101B851EA6A4A0F19
:100DF000E96E020EEA22DFCFEFFF0101CC6B0101A9
:100E0000B82B01D013D0400E0101B85D02E1010101
:100E1000B86B0101B9510101B85D02E10D8609D03D
:100E2000010EDB5003E01CD9010EDB6A0101992B96
:100E3000A8D70401400E196F400E040118170401D1
:100E4000187D880E040118130D5001E181D00DA00A
:100E500010D06F0E2A6E400E2B6E2C6A2AC0E6FF51
:100E60002BC0E6FF2CC0E6FF67EC21F0E552E5520F
:100E7000E5520DA210D0690E2A6E400E2B6E2C6A20
:100E80002AC0E6FF2BC0E6FF2CC0E6FF67EC21F08E
:100E9000E552E552E5520DA410D04D0E2A6E400EDB
:100EA0002B6E2C6A2AC0E6FF2BC0E6FF2CC0E6FFA3
:100EB00067EC21F0E552E552E5520DA610D0310E57
:100EC0002A6E400E2B6E2C6A2AC0E6FF2BC0E6FF6E
:100ED0002CC0E6FF67EC21F0E552E552E5520DA883
:100EE00010D0120E2A6E400E2B6E2C6A2AC0E6FF1E
:100EF0002BC0E6FF2CC0E6FF67EC21F0E552E5527F
:100F0000E5520DAA00D00DAC10D0F10E2A6E3F0EA6
:100F10002B6E2C6A2AC0E6FF2BC0E6FF2CC0E6FF32
:100F200067EC21F0E552E552E5520DAE10D0D80E37
:100F30002A6E3F0E2B6E2C6A2AC0E6FF2BC0E6FFFE
:100F40002CC0E6FF67EC21F0E552E552E5520D6A50
:100F500035D8020EE15C02E2E16AE552E16EE5524B
:100F6000E7CFD9FF1200D9CFE6FFE1CFD9FF0101CA
:100F7000B651EA6A000FE96E020EEA22FE0EDBCFDE
:100F8000EFFF0101B62B4A0E0101B65D02E101013E
:100F9000B66B0101B7510101B65D01E10D84FE0E92
:100FA000DBCF2AF02B6A2ABE2B682AC0F3FF2BC0A6
:100FB000F4FF00D0E552E7CFD9FF1200D9CFE6FF0A
:100FC000E1CFD9FFE65201019A5145E1060E010138
:100FD000C85D41E36D50020B3EE10101B6510101D4
:100FE000B75D39E00101B7510101D880B6551AE269
:100FF0000101B7510101B65DDF6E0101B751010179
:101000009B6F9C6B000E01019B27020E01019C232C
:10101000DFCF9FF10101A06B0101010E9A6FB6C1F4
:10102000B7F119D04A0E0101D880B755DF6E010122
:10103000B75101019B6F9C6B000E01019B27020EB3
:1010400001019C23DFCF9FF10101A06B0101010E83
:101050009A6F0101B76BE552E552E7CFD9FF120055
:10106000D9CFE6FFE1CFD9FF040EE126DE6ADD6AC3
:10107000020EDB6A030EDB6A0101B951EA6A4A0F0C
:10108000E96E020EEA22EF50E66EE66A60EC22F0AC
:10109000E552E552020EF3CFDBFF0101B92B400E02
:1010A0000101B95D02E10101B96B020EDB50DE6E98
:1010B000DD6A0101B951EA6A4A0FE96E020EEA22BD
:1010C000EF502C0835E00101B951EA6A4A0FE96E88
:1010D000020EEA22EF500D082BE00101B951EA6A35
:1010E0004A0FE96E020EEA22EF50E66EE66A60EC05
:1010F00022F0E552E552030EF3CFDBFF0101B92BDD
:10110000400E0101B95D02E10101B96B020EDBCFB6
:101110002CF02CC02DF02C6A030EDB5000012C2487
:101120002A6E000E2D202B6E2AC0DEFF2BC0DDFFA5
:10113000000EDBCF1EF0010EDBCF1FF0490E1E1894
:1011400002E1430E1F1801E1D7D0490E1E1802E13B
:10115000520E1F1801E1CDD0490E1E1802E1530EA8
:101160001F1801E1C3D0530E1E1802E1430E1F18D1
:1011700001E1B9D0530E1E1802E1520E1F1801E111
:10118000AFD0530E1E1802E1530E1F1801E1A5D077
:10119000530E1E1802E1420E1F1801E19BD0430EB0
:1011A0001E1802E1420E1F1801E191D0430E1E18D5
:1011B00002E1520E1F1801E187D04F0E1E1802E106
:1011C000420E1F1801E17DD0570E1E1802E14D0E90
:1011D0001F1875E0520E1E1802E14D0E1F186DE02B
:1011E000440E1E1802E1500E1F1865E04F0E1E1827
:1011F00002E1500E1F185DE0490E1E1802E1500E6C
:101200001F1855E0580E1E1802E1540E1F184CE02E
:10121000540E1E1801E11F5045E0410E1E1801E159
:101220001F503EE0560E1E1801E11F5037E0490ED8
:101230001E1801E11F5030E04F0E1E1801E11F5033
:1012400029E0550E1E1802E1430E1F1821E0580E2A
:101250001E1802E1430E1F1818E0430E1E1801E18C
:101260001F5011E0520E1E1801E11F500AE0580EE7
:101270001E1802E1520E1F1801E041D0CCEC0DF017
:101280007DD0B3D87BD036D979D0CEEC0DF076D0E6
:10129000B0D874D08CD972D0BDD970D0D6D96ED018
:1012A000E5D96CD0E6D86AD0CAEC0DF067D051DB36
:1012B00065D0D7DB63D0B1DA61D06EDA5FD037DAD0
:1012C0005DD0BCEC0EF05AD0D0EC0DF057D075ECE0
:1012D0000EF054D003EC10F051D0BFEC10F04ED013
:1012E000C2EC10F04BD0C5EC10F048D0C8EC10F0B8
:1012F00045D0CBEC10F042D0CEEC10F03FD0030E36
:10130000DB501AE1020EDBCFE6FFE66A020EDBCF0E
:10131000E6FFE66AB50E2A6E3F0E2B6E2C6A2AC0D7
:10132000E6FF2BC0E6FF2CC0E6FF67EC21F02D6E38
:10133000070EE15E2D5021D0030EDBCFE6FFE66AFB
:10134000020EDBCFE6FFE66A030EDBCFE6FFE66ABE
:10135000020EDBCFE6FFE66A8D0E2A6E3F0E2B6E85
:101360002C6A2AC0E6FF2BC0E6FF2CC0E6FF67EC24
:1013700021F02D6E0B0EE15E2D5000D00101B95110
:10138000EA6A4A0FE96E020EEA22EF500D080DE0FC
:101390000D500BE1520E2A6E2B6ADF502A1803E122
:1013A000DE52DD502B1801E00D8EB8C1B9F1040EEC
:1013B000E15C02E2E16AE552E16EE552E7CFD9FF76
:1013C00012000101BE5110E08C0E2A6E450E2B6EEC
:1013D0002C6A2AC0E6FF2BC0E6FF2CC0E6FF67ECB4
:1013E00021F0E552E552E5521200C4EC05F0E9DFC8
:1013F0001200D9CFE6FFE1CFD9FF030EE126010E9F
:10140000E66ED1EC10F0E5521D50DF6E020EE66E76
:10141000D1EC10F0E552DE521DC0DEFF1EC0DDFF34
:10142000DD520D5001E01BD0DF0418E1D950010F4F
:10143000E96EDACFEAFFEE50ED100BE0010E2A6EF6
:101440002B6A010EDB502A1803E1020EDB502B1829
:1014500004E1010EDBCFBEF101D00D8CB2DF030E33
:10146000E15C02E2E16AE552E16EE552E7CFD9FFC5
:101470001200D9CFE6FFE1CFD9FF030EE126020E1D
:10148000DB6A030EE66ED1EC10F0E5521DC000F0F1
:101490001EC001F0010EE66ED1EC10F0E552020E16
:1014A0001DC0DBFF0D5001E01BD0020EDB500CE134
:1014B0000050011003E1026A036A05D0CA8400C02B
:1014C00002F001C003F00BD00050011003E1076AE5
:1014D000086A05D0CA8400C007F001C008F071DFB7
:1014E000030EE15C02E2E16AE552E16EE552E7CF0C
:1014F000D9FF1200D9CFE6FFE1CFD9FF040EE126D4
:10150000010EE66ED1EC10F0E5521D50DF6E010EBB
:10151000E66ED1EC10F0E552010E1DC0DBFF010EAE
:10152000E66ED1EC10F0E552020E1DC0DBFF010E9D
:10153000E66ED1EC10F0E552030E1DC0DBFF0D503E
:1015400001E02BD0DF50926E010EDB50936E020E45
:10155000DB50946E030EDB500D0805E20D0EF36EAA
:10156000030EF3CFDBFF030EDB5005E10F0EC16E60
:10157000C2900C6A11D00C6AC26A030EDBCFE6FF80
:101580000F0EE552D880E754C16EBE0EC06EC28009
:10159000030EDB500C6ECA8414DF040EE15C02E221
:1015A000E16AE552E16EE552E7CFD9FF1200D9CFEB
:1015B000E6FFE1CFD9FF030EE126010EE66ED1EC86
:1015C00010F0E5521D50DF6E010EE66ED1EC10F00A
:1015D000E552010E1DC0DBFF010EE66ED1EC10F0EE
:1015E000E552020E1DC0DBFF0D5001E009D0DF50B7
:1015F000896E010EDB508A6E020EDB508B6EE1DECF
:10160000030EE15C02E2E16AE552E16EE552E7CFEA
:10161000D9FF12008250E66EE66A8150E66EE66AF5
:101620008050E66EE66A7A0E2A6E3F0E2B6E2C6AAA
:101630002AC0E6FF2BC0E6FF2CC0E6FF67EC21F0D6
:101640002D6E090EE15E2D501200940E2A6E450E8D
:101650002B6E2C6A2AC0E6FF2BC0E6FF2CC0E6FFEB
:1016600067EC21F0E552E552E5521200D9CFE6FFD2
:10167000E1CFD9FFE652DF6A780E2A6E3F0E2B6E5D
:101680002C6A2AC0E6FF2BC0E6FF2CC0E6FF67EC01
:1016900021F0E552E552E552DF6A0C50DF5C32E2A0
:1016A000DFCF2AF02B6A2ABE2B68060E2B02F3CF5F
:1016B0002BF0060E2A02F3CF2AF0F4502B26000E50
:1016C0002A26010E2B220A50020D2A50F324E96E1D
:1016D0002B50F420EA6EEECFE6FFEFCFE6FF720E5E
:1016E0002C6E3F0E2D6E2E6A2CC0E6FF2DC0E6FF3D
:1016F0002EC0E6FF67EC21F02F6E050EE15E2F5045
:10170000DF2ACBD7910E2A6E450E2B6E2C6A2AC08B
:10171000E6FF2BC0E6FF2CC0E6FF67EC21F0E552A8
:10172000E552E552E552E552E7CFD9FF1200D9CF95
:10173000E6FFE1CFD9FF030EE126030EE66ED1EC02
:1017400010F0E5521DC0DEFF1EC0DDFF010EE66E8B
:10175000D1EC10F0E552020E1DC0DBFF0D5001E090
:1017600011D0DECF2AF0DDCF2BF0000E2A5C100E58
:101770002B5807E2DECFE9FFDDCFEAFF020EDBCF19
:10178000EFFF1FDE030EE15C02E2E16AE552E16E6B
:10179000E552E7CFD9FF1200D9CFE6FFE1CFD9FF5D
:1017A000030EE126030EE66ED1EC10F0E5521DC0EB
:1017B000DEFF1EC0DDFF0D5001E025D0DECF2AF098
:1017C000DDCF2BF0000E2A5C100E2B5807E2DECF87
:1017D000E9FFDDCFEAFF020EEFCFDBFF020EDBCF2A
:1017E000E6FFE66A680E2A6E3F0E2B6E2C6A2AC050
:1017F000E6FF2BC0E6FF2CC0E6FF67EC21F02D6E64
:10180000050EE15E2D50030EE15C02E2E16AE55255
:10181000E16EE552E7CFD9FF1200D9CFE6FFE1CF65
:10182000D9FF030EE126050EE66ED1EC10F0E5526D
:101830001D50DF6E010EE66ED1EC10F0E552010E88
:101840001DC0DBFF010EE66ED1EC10F0E552020E7A
:101850001DC0DBFF0D5001E072D0020EDB5001080D
:1018600002E20D8C6CD0010EDB50070802E20D8CF9
:1018700066D0410E2A6EDF502A5C1CE1020EDB505E
:101880000DE1010EF36E010EDB5004E0D890F3364B
:10189000E806FCE1F350E81C92160BD0010EF36E43
:1018A000010EDB5004E0D890F336E806FCE1F3507B
:1018B000921244D0420E2A6EDF502A5C1CE1020EC6
:1018C000DB500DE1010EF36E010EDB5004E0D89009
:1018D000F336E806FCE1F350E81C93160BD0010E3A
:1018E000F36E010EDB5004E0D890F336E806FCE11D
:1018F000F350931223D0430E2A6EDF502A5C1CE172
:10190000020EDB500DE1010EF36E010EDB5004E020
:10191000D890F336E806FCE1F350E81C94160BD09F
:10192000010EF36E010EDB5004E0D890F336E806AA
:10193000FCE1F350941202D00D8C01D042DD030E75
:10194000E15C02E2E16AE552E16EE552E7CFD9FFE0
:101950001200D9CFE6FFE1CFD9FF030EE126020E38
:10196000DB6A050EE66ED1EC10F0E5521D50DF6E1D
:10197000010EE66ED1EC10F0E552010E1DC0DBFF4A
:101980000D5001E064D0010EDB50070802E20D8C1F
:101990005ED0410E2A6EDF502A5C10E1010EF36E1C
:1019A000010EDB5004E0D890F336E806FCE1F3507A
:1019B0008014E76E020EE7CFDBFF2CD0420E2A6EBA
:1019C000DF502A5C10E1010EF36E010EDB5004E0E3
:1019D000D890F336E806FCE1F3508114E76E020E6E
:1019E000E7CFDBFF17D0430E2A6EDF502A5C10E1F1
:1019F000010EF36E010EDB5004E0D890F336E806DA
:101A0000FCE1F3508214E76E020EE7CFDBFF02D059
:101A10000D8C1DD0020EDB5005E0010EF36E020EA0
:101A2000F3CFDBFF020EDBCFE6FFE66A5F0E2A6E26
:101A30003F0E2B6E2C6A2AC0E6FF2BC0E6FF2CC09F
:101A4000E6FF67EC21F02D6E050EE15E2D50030ED2
:101A5000E15C02E2E16AE552E16EE552E7CFD9FFCF
:101A60001200D9CFE6FFE1CFD9FF030EE126050E24
:101A7000E66E97DBE5521D50DF6E010EE66E91DBE0
:101A8000E552010E1DC0DBFF010EE66E8ADBE5525A
:101A9000020E1DC0DBFF0D5001E072D0020EDB50C4
:101AA000010802E20D8C6CD0010EDB50070802E247
:101AB0000D8C66D0410E2A6EDF502A5C1CE1020EAE
:101AC000DB500DE1010EF36E010EDB5004E0D89007
:101AD000F336E806FCE1F350E81C89160BD0010E42
:101AE000F36E010EDB5004E0D890F336E806FCE11B
:101AF000F350891244D0420E2A6EDF502A5C1CE15A
:101B0000020EDB500DE1010EF36E010EDB5004E01E
:101B1000D890F336E806FCE1F350E81C8A160BD0A7
:101B2000010EF36E010EDB5004E0D890F336E806A8
:101B3000FCE1F3508A1223D0430E2A6EDF502A5C58
:101B40001CE1020EDB500DE1010EF36E010EDB50C5
:101B500004E0D890F336E806FCE1F350E81C8B165D
:101B60000BD0010EF36E010EDB5004E0D890F3367B
:101B7000E806FCE1F3508B1202D00D8C01D021DC81
:101B8000030EE15C02E2E16AE552E16EE552E7CF65
:101B9000D9FF120016DC120014DC120012DC120055
:101BA000D9CFE6FFE1CFD9FF040EE126050EE66EA0
:101BB000F8DAE5521D50DF6E010EE66EF2DAE552FC
:101BC000010E1DC0DBFF030EE66EEBDAE552020EDE
:101BD0001DC0DBFF030E1EC0DBFF0D5001E07BD0FC
:101BE000D950020FE96EDACFEAFF720ED880EE54B8
:101BF0002E0EED5402E20D8C6ED0D950020FE96E1C
:101C0000DACFEAFFEE50ED101FE02D682E682F6A44
:101C10002D0EE76E020EDBCF30F0030EDBCF31F07E
:101C2000E7503026000E3122326A30502D5C2A6E89
:101C300031502E582B6E32502F582C6E020E2AC067
:101C4000DBFF030E2BC0DBFF010EDB50070802E2B7
:101C50000D8C41D0410E2A6EDF502A5C02E1DF6A12
:101C600012D0420E2A6EDF502A5C03E1080EDF6EAE
:101C70000AD0430E2A6EDF502A5C03E1100EDF6E9D
:101C800002D00D8C28D0010EDB50DF24E96EEA6A09
:101C9000D890E936EA36690EE926010EEA22020EEC
:101CA000DBCFEEFF030EDBCFEDFF010EDB50DF24B9
:101CB000EA6A510FE96E010EEA22EF040AE1010E11
:101CC000DB50DF24EA6A510FE96E010EEA22020EB0
:101CD000EF6EE1EC09F0040EE15C02E2E16AE5522C
:101CE000E16EE552E7CFD9FF1200D9CFE6FFE1CF91
:101CF000D9FF050EE126010EE66E53DAE5521D50BE
:101D0000DF6E010EE66E4DDAE552020E1DC0DBFFFE
:101D1000010EE66E46DAE552030E1DC0DBFF010E32
:101D2000E66E3FDAE552010E1DC0DBFF010EE66EE6
:101D300038DAE552040E1DC0DBFF0D5001E012D071
:101D4000DFCFB1F1020EDBCFB3F1010EDBCFB2F189
:101D5000030EDBCFB4F1040EDBCFB5F1B1C189FFC7
:101D6000E1EC09F0050EE15C02E2E16AE552E16EA8
:101D7000E552E7CFD9FF1200D9CFE6FFE1CFD9FF77
:101D8000040EE126030EDB6A0101B951EA6A4A0F2B
:101D9000E96E020EEA22EF502C081DE00101B95154
:101DA000EA6A4A0FE96E020EEA22EF50E66EE66A30
:101DB000380E2A6E3F0E2B6E2C6A2AC0E6FF2BC00F
:101DC000E6FF2CC0E6FF67EC21F02D6E050EE15E0C
:101DD0002D500D8A0ED10101B92B400E0101B95DC4
:101DE00002E10101B96BB1C189FF0101B21D891482
:101DF0002A6E891C0101B2152A10E76E010EE7CF89
:101E0000DBFF0101B951EA6A4A0FE96E020EEA22CC
:101E1000EF500D0801E1EBD00101B951EA6A4A0F18
:101E2000E96E020EEA22EF50E66EE66A60EC22F0FE
:101E3000E552E552020EF3CFDBFF300EF36E020ED9
:101E4000DBCFF4FFF350F45C0FE3020EDB503908F4
:101E50000BE3300E2A6E020EDBCFE7FF2A50E75E5F
:101E6000020EE7CFDBFF19D0410EF36E020EDBCF7F
:101E7000F4FFF350F45C0FE3020EDB5046080BE373
:101E8000370E2A6E020EDBCFE7FF2A50E75E020E06
:101E9000E7CFDBFF02D00D8CACD0020EDB38F00BAD
:101EA000DF6E0101B92B400E0101B95D02E10101B4
:101EB000B96B0D0E2A6E0101B951EA6A4A0FE96E3B
:101EC000020EEA22EF502A5C02E10D8892D0010155
:101ED000B951EA6A4A0FE96E020EEA22EF50E66E45
:101EE000E66A60EC22F0E552E552020EF3CFDBFF2A
:101EF000300EF36E020EDBCFF4FFF350F45C0FE311
:101F0000020EDB5039080BE3300E2A6E020EDBCFD7
:101F1000E7FF2A50E75E020EE7CFDBFF19D0410E44
:101F2000F36E020EDBCFF4FFF350F45C0FE3020E0E
:101F3000DB5046080BE3370E2A6E020EDBCFE7FFBD
:101F40002A50E75E020EE7CFDBFF02D00D8C51D0A6
:101F5000020EDB50DF24DF6E0101B92B400E0101C0
:101F6000B95D02E10101B96BDF508A6E010EDB50F1
:101F7000896E0101B55105E0B5C1E6FF01EC23F022
:101F8000E552B1C189FF0101B45130E0030EB4C183
:101F9000DBFF0101B1510101B3152A6E0101B351FB
:101FA00080142A5C0BE1030EDB5008E00000000007
:101FB000000000000000030EDB06EBD7030EB4C1E7
:101FC000DBFF0101B1510101B3152A6E0101B351CB
:101FD00080142A5C0BE0030EDB5008E000000000D8
:101FE000000000000000030EDB06EBD70AD7E1EC8F
:101FF00009F0040EE15C02E2E16AE552E16EE552AD
:10200000E7CFD9FF1200D9CFE6FFE1CFD9FF050E08
:10201000E126030EDB6A040EDB6A010EE66EC1D810
:10202000E552040E1DC0DBFF040EDB5004E0040E7D
:10203000DB50380802E20D8C98D00101B951EA6AF0
:102040004A0FE96E020EEA22EF502C081DE0010152
:10205000B951EA6A4A0FE96E020EEA22EF50E66EC3
:10206000E66A380E2A6E3F0E2B6E2C6A2AC0E6FFF7
:102070002BC0E6FF2CC0E6FF67EC21F02D6E050EAD
:10208000E15E2D500D8A71D00101B92B400E010186
:10209000B95D02E10101B96BB1C189FF0101B21D56
:1020A00089142A6E891C0101B2152A10E76E010EEF
:1020B000E7CFDBFF040EDB5056E00101B951EA6ABD
:1020C0004A0FE96E020EEA22EFCFDFFF0101B92BC2
:1020D000400E0101B95D02E10101B96B040EDB069E
:1020E000DF508A6E010EDB50896E0101B55105E0AB
:1020F000B5C1E6FF01EC23F0E552B1C189FF010152
:10210000B45130E0030EB4C1DBFF0101B151010154
:10211000B3152A6E0101B35180142A5C0BE1030E42
:10212000DB5008E000000000000000000000030E8B
:10213000DB06EBD7030EB4C1DBFF0101B151010196
:10214000B3152A6E0101B35180142A5C0BE0030E13
:10215000DB5008E000000000000000000000030E5B
:10216000DB06EBD7A7D7E1EC09F0050EE15C02E254
:10217000E16AE552E16EE552E7CFD9FF1200E1ECEA
:1021800009F01200E1EC09F01200E1EC09F0120094
:10219000E1EC09F01200E1EC09F01200E1EC09F0C9
:1021A0001200D9CFE6FFE1CFD9FF040EE126030EDE
:1021B000DB6A0D0E2A6E0101B951EA6A4A0FE96E17
:1021C000020EEA22EF502A5C05E10D881D6A1E6AA4
:1021D0001F6A93D10101B951EA6A4A0FE96E020EF2
:1021E000EA22EF502C0820E00101B951EA6A4A0FB7
:1021F000E96E020EEA22EF50E66EE66A380E2A6EAB
:102200003F0E2B6E2C6A2AC0E6FF2BC0E6FF2CC0C7
:10221000E6FF67EC21F02D6E050EE15E2D500D8A74
:102220001D6A1E6A1F6A69D10101B92B400E0101A6
:10223000B95D02E10101B96B2D0E2A6E0101B951A0
:10224000EA6A4A0FE96E020EEA22EF502A5C28E1A0
:10225000040E2B6EFE0EDB502B5C22E0050E2C6E66
:10226000FE0EDB502C5C1CE0FE0EDB0406E0030ED1
:102270002A6EFE0EDB502A5C06E10D8C1D6A1E6A7A
:102280001F6A3BD10DD0010EF36E030EF3CFDBFFBF
:102290000101B92B400E0101B95D02E10101B96BE9
:1022A000040E2A6EFE0EDB502A5C11E0050E2B6E2A
:1022B000FE0EDB502B5C0BE0050EE66ED9CFE6FF81
:1022C000DACFE6FF24D9E552E552E5523AD00101D2
:1022D000B951EA6A4A0FE96E020EEA22EFCF2AF0FC
:1022E0002B6A2C6A2AC0DFFF010E2BC0DBFF020E17
:1022F0002CC0DBFF050E2A6EFE0EDB502A5C19E1B6
:10230000000EDBCFE6FF010EDBCFE6FF60EC22F034
:10231000E552E552F3CF2AF0F4CF2BF02C6A2BBE16
:102320002C682AC0DFFF010E2BC0DBFF020E2CC081
:10233000DBFF0101B92B400E0101B95D02E1010192
:10234000B96B030EDB5021E0DFCF2AF0010EDBCFAB
:102350002BF0020EDBCF2CF02268236824682AC001
:102360001DF02BC01EF02CC01FF03BEC20F01AC05B
:102370002AF01BC02BF01CC02CF02AC0DFFF010E7E
:102380002BC0DBFF020E2CC0DBFFFE0EDB5026E174
:10239000DFCF2AF0010EDBCF2BF0020EDBCF2CF0CB
:1023A0002C34000E2C1807E6D8807F0E2A54000E1D
:1023B0002B54000E2C5401E28CD0D9CFE9FFDACF98
:1023C000EAFF020ED880EB50FF0A06E6800EEE5CB4
:1023D000FF0EEE58FF0EEF5801E27BD0FE0EDB043D
:1023E00024E1DFCF2DF0010EDBCF2EF0020EDBCF8C
:1023F0002FF02F34000E2F1807E6D880FF0E2D5433
:10240000000E2E54000E2F5464E3D9CFE9FFDACF2B
:10241000EAFF020ED890EB50000A06E6000EEE5CD2
:10242000000EEE58000EEF5854E3020E306EFE0E12
:10243000DB50305C24E1DFCF31F0010EDBCF32F036
:10244000020EDBCF33F03334000E331807E6D880AA
:10245000FF0E31547F0E3254000E33543AE3D9CF7D
:10246000E9FFDACFEAFF020ED880EB50FF0A06E65A
:10247000000EEE5C800EEE58FF0EEF582AE3030EBE
:10248000346EFE0EDB50345C29E1DFCF35F0010EF7
:10249000DBCF36F0020EDBCF37F03734000E3718C3
:1024A00007E6D880FF0E3554FF0E3654000E375421
:1024B00010E3D9CFE9FFDACFEAFF020ED890EB5054
:1024C000000A06E6000EEE5C000EEE58000EEF5815
:1024D00005E20D8C1D6A1E6A1F6A0FD0DFCF2AF03D
:1024E000010EDBCF2BF0020EDBCF2CF02AC01DF04B
:1024F0002BC01EF02CC01FF000D0040EE15C02E2E5
:10250000E16AE552E16EE552E7CFD9FF1200D9CF7B
:10251000E6FFE1CFD9FF020EE126FD0EDBCFE9FF9A
:10252000FE0EDBCFEAFFEE6AEE6AEE6A010EDB6AB0
:10253000FC0EDB50F36E010EDBCFF4FFF350F45CC6
:1025400055E20101B951EA6A4A0FE96E020EEA2228
:10255000EFCFDFFF300EDF5C44E3DF50390841E3AB
:10256000FD0EDBCFE9FFFE0EDBCFEAFFEECF2DF055
:10257000EECF2EF0EFCF2FF00A0E226E236A246AE0
:102580002DC01DF02EC01EF02FC01FF03BEC20F020
:102590001AC02DF01BC02EF01CC02FF0300EDF5CD7
:1025A000306E316A326A2D5030242A6E2E5031201E
:1025B0002B6E2F5032202C6EFD0EDBCFE9FFFE0E6E
:1025C000DBCFEAFF2AC0EEFF2BC0EEFF2CC0EEFFF0
:1025D0000101B92B400E0101B95D02E10101B96BA6
:1025E00002D0000E05D0010EDB2AA2D7010E00D0CA
:1025F0002A6E020EE15C02E2E16AE552E16E2A50C7
:10260000E552E7CFD9FF12000650E66EE66A2C0EBF
:102610002A6E3F0E2B6E2C6A2AC0E6FF2BC0E6FF07
:102620002CC0E6FF67EC21F02D6E050EE15E2D500B
:1026300012000101C85108E0010E2A6E6D50020B14
:1026400001E0010E2A5C22E10101CD07000ECE5B04
:102650000101CF510EE10101CD51CE1109E18B8075
:102660000101D00ECD6F070ECE6F0101010ECF6FAD
:102670000CD00101CD51CE1108E18B900101D00E9B
:10268000CD6F070ECE6F0101CF6B5DD00101C80584
:102690000CE0020E0101C85D08E0030E0101C85DF7
:1026A00004E0050E0101C85D02E18B804CD0060EEE
:1026B0000101C85D48E10101CD07000ECE5B0101BB
:1026C000CF510EE10101CD51CE1109E18B80010105
:1026D000100ECD6F270ECE6F0101010ECF6F33D0DC
:1026E0000101CF050EE10101CD51CE1109E18B9021
:1026F0000101100ECD6F270ECE6F0101020ECF6FBC
:1027000022D0020E0101CF5D0EE10101CD51CE11AB
:1027100009E18B800101A00ECD6F860ECE6F010105
:10272000030ECF6F10D0030E0101CF5D0CE301014A
:10273000CD51CE1108E18B900101100ECD6F270E07
:10274000CE6F0101CF6B120082B403D0010E03D013
:0827500002D0000E00D01200BF
:08275800E8EC18F0FB0EDBCFEA
:10276000F3FFDB06F35000090AE036EC19F0FA0E2D
:10277000A1EC19F0F3E12B1CF1E1010E01D0000EE8
:1027800017EF19F0E8EC18F03B0EE12402E3E168E2
:10279000E652E16E010EDB6A020EDB6AF90EDBCF58
:1027A000F6FFFA0EDBCFF7FFFB0EDBCFF8FF0800DA
:1027B000F550DF6EDF5002E13BEF18F0250EDF5CD5
:1027C00002E02EEF18F0030EDB6A040EDB6A050E42
:1027D000DB6A060EDB6A070EDB6A50EC18F02D0E82
:1027E000DF5C0CE02B0EDF5C09E0200EDF5C06E016
:1027F000230EDF5C03E0300EDF5C1AE1DF50300AAD
:1028000014E0130A0FE0030A0AE00B0A05E0060AC7
:10281000E4E1030EDB80E1D7030EDB82DED7030E9B
:10282000DB84DBD7030EDB86D8D7030EDB88D5D756
:102830002A0EDF5C1BE14CEC18F09AEC18F010E06B
:10284000030EDB801E681F68130EDBCF23F0140E0F
:10285000DBCF24F084EC20F0040E1CC0DBFF03D09F
:10286000130E83EC18F050EC18F00BD0090EDB6A55
:10287000F1EC18F003E065EC19F0FAD7090E83ECDF
:1028800018F0030EDBB0DB982E0EDF5C1BE150EC82
:1028900018F02A0EDF5C0BE14CEC18F09AEC18F003
:1028A00003E1130ED5EC18F050EC18F00BD0090E24
:1028B000DB6AF1EC18F003E065EC19F0FAD7090EC9
:1028C000D5EC18F0680EDF5C07E150EC18F0680EEC
:1028D000DF5C1DE1030E18D0740EDF5C17E07A0E8A
:1028E000DF5C14E0480EDF5C06E0540EDF5C03E0C2
:1028F0005A0EDF5C02E1020E07D06C0EDF5C03E0D3
:102900006A0EDF5C04E1010E28EC19F0C9DBDF5030
:102910006E0A01E17FD31E0A01E192D1200A01E192
:102920008FD13F0A01E149D11A0A01E146D10D0ACE
:1029300001E143D1200A01E140D13A0A01E13DD150
:10294000200A01E13AD1260A01E135D10D0A01E15F
:1029500032D11A0A01E1D9D0200A4AE0300A1FE038
:10296000460A0EE0250A01E083D3D950F90FE96E3B
:10297000FF0EDA20EA6E010EEE5E000EEE5AEE5AFF
:1029800036EC19F0250EE66E95DB03E12B1C01E118
:1029900069D332EC19F001E26BD3DB2A69D3080E5C
:1029A000DB6A040EDB50010806E2040EDB04FAECDD
:1029B00018F0DB508BDB080EDB5009E0030EDB5018
:1029C000010B05E172DB01E04DD3080EDB6A64DB2D
:1029D000EFCFDFFFAAEC19F003E12B1C01E142D39A
:1029E00032EC19F001E3DB2A60DB01E141D33AD399
:1029F000070EDB5002080FE176EC19F0030E3DECF8
:102A000019F00E0EEECFDBFF0F0EEECFDBFF100E38
:102A1000EECFDBFF20D0F70EDBCF2DF0F80EDBCFB3
:102A20002EF0020E2D5E000E2E5AF70E2DC0DBFF8B
:102A3000F80E2EC0DBFF2DC0E9FF2EC0EAFF2DEC03
:102A400019F02C6A0E0E2AC0DBFF0F0E2BC0DBFF25
:102A5000100E2CC0DBFF0E0EDBCFE6FF0F0EDBCF20
:102A6000E6FF100EDBCFE6FF3BEC22F0E552E5522D
:102A7000E552130E1DC0DBFF140E1EC0DBFF060E59
:102A8000DB5005E0130E71EC19F001E26ADB95EC06
:102A900019F002E2130E37DB58EC19F006E0040ED1
:102AA00071EC19F002E2050E2EDB030EDBB005D04F
:102AB000FCDA01E0D7D2080EDB6A090EDB6A0E0EE3
:102AC000DBCFF6FF0F0EDBCFF7FF100EDBCFF8FFEB
:102AD0000800F550DF6EDF5014E09BEC19F011E2B6
:102AE000AAEC19F003E12B1C01E1BCD2BBDB01E332
:102AF000DB2A090EDB2AD9500E0FE96E000ECBDB64
:102B0000E7D7D3DA01E1B4D2ADD2C6DA110EEECFF7
:102B1000DBFF120EEDCFDBFF110EDBCFE6FF120E57
:102B2000DBCFE6FF2DEC22F0E552E552130EF3CF9A
:102B3000DBFF140EF4CFDBFF060EDB5004E0130EB8
:102B4000D0DB01E20EDB95EC19F002E2130EDBDACA
:102B5000AFDB05E0040EC5DB02E2050ED4DA030E9E
:102B6000DBB005D0A2DA01E07DD2080EDB6A090EE7
:102B7000DB6A110EDBCFE9FF120EDBCFEAFFEFCFEE
:102B8000DFFFDF5014E0D7DB12E2E4DB03E12B1CB4
:102B900001E168D267DB01E3DB2A090EDB2A110EB3
:102BA000DB2ADBCFE9FF120EE8E3DB2AE6D77DDA8A
:102BB00001E15ED257D2030EDB8E070EDB0410E17B
:102BC00095DB040E5ADB0A0EEECFDBFF0B0EEECFC9
:102BD000DBFF0C0EEECFDBFF0D0EEECFDBFF6CD07C
:102BE000070EDB5003082CE1030EDBAE0DD0B2DA8A
:102BF000020E76DAEFCF2AF02B6A2C6A2D6A2AAE03
:102C000039D02B682C6835D0F70EDBCF2BF0F80EBF
:102C1000DBCF2CF0020E2B5E000E2C5AF70E2BC0D1
:102C2000DBFFF80E2CC0DBFF2BC0E9FF2CC0EAFF56
:102C3000EFCF2AF00A0E2AC0DBFF0B0EDB6A38D07A
:102C4000070EDB50020809E1030EDBAE04D059DBAE
:102C50002CAE10D00ED055DB0DD0030EDBAE12D053
:102C600079DA020E3DDAF9DA2C6A2D6A2BAE02D03F
:102C70002C682D68E2DA0C0E2CC0DBFF0D0E2DC087
:102C8000DBFF1AD0F70EDBCF2CF0F80EDBCF2DF0E8
:102C9000020E2C5E000E2D5AF70E2CC0DBFFF80E34
:102CA0002DC0DBFF2CC0E9FF2DC0EAFFD6DAC5DA64
:102CB0000C0EDB6A0D0EDB6A060EDB5005E1010E21
:102CC000F36E050EF3CFDBFF150EDB6A160EDB6A23
:102CD000D950370F2A6E000EDA202B6E390E2AC01B
:102CE000DBFF3A0E2BC0DBFF380EDB6A080EDB6A17
:102CF0000A0EAEDADF50780A12E0200A10E0280A45
:102D00000CE0200A0AE03F0A06E00D0A02E0200A71
:102D100008E1020E05D0080E03D0080EDF26100EC3
:102D200097DA030EDBBE02D0DB92DB94DB50800B24
:102D300024E08ADAD890030EEB50000A08E6000E71
:102D4000EE5C000EEE58000EEE58000EEE5815E246
:102D500013DA2168226823682468F5EC21F00A0E52
:102D600018C0DBFF0B0E19C0DBFF0C0E1AC0DBFF17
:102D70000D0E1BC0DBFF2D0E08D0030EDBA202D010
:102D80002B0E03D0DBA408D0200EF36E170EF3CF6A
:102D9000DBFF150EDB2A02D0170EDB6A050EDB50B7
:102DA00003E1B7D901E189D0180E2A6E460E2B6EC9
:102DB000000E2C6E070EDBCF2DF02E6A2F6A306AC4
:102DC0002DC021F02EC022F02FC023F030C024F0FF
:102DD000D3D986EC22F02A501824F36E2B501920F8
:102DE000F46E2C501A20F86EF4CFF7FFF3CFF6FFF5
:102DF0000800090EF5CFDBFF580EDF5C0FE1610E16
:102E0000F36E090E7BD90AE3200E2A6E090EDBCF82
:102E1000E7FF2A50E75E090EE7CFDBFF070EDBCFA7
:102E20002AF02B6A2C6A2D6A0FDA2AC021F02BC0F7
:102E300022F02CC023F02DC024F0EECF1CF0EECFFA
:102E40001DF0EECF1EF0EFCF1FF086EC22F01FC07A
:102E5000EDFF1EC0EDFF1DC0EDFF1CC0EFFF390EE2
:102E6000DBCFE9FFDB063A0EDBCFEAFF01E2DB0650
:102E7000090EDBCFEFFF150EDB2A4BD995E1030ED0
:102E8000DBA61DD06F0EDF5C06E1C1D918E3150E7D
:102E9000DB285BDA14D0780EDF5C09E0580EDF5CCB
:102EA00006E0620EDF5C03E0420EDF5C08E1020E2A
:102EB000F36E160EF3CFDBFF02D0150EDB6A030EA6
:102EC000DB50100B0EE0040EDBCF2AF0050EDB50BA
:102ED000D8802A5406E2060EDB5003E1040EDB50D4
:102EE00034DA95D90AE2050EDBCFE7FF150EDB5089
:102EF000E75E050EE7CFDBFF02D0050EDB6A040EAE
:102F0000DBCF2AF0160E45D9D8802A5414E2160ECB
:102F1000DBCFE6FF150EDBCFE6FF040EDBCFE6FFCF
:102F2000050EDB50E552E75CE552D880E754E552E8
:102F3000D880E7545FD9030EDB50010B0BE1080E7C
:102F4000DB5008E0B2D801E08DD0080EDB50BED8CF
:102F5000080EDB6A170EDB5007E088D9170EF1D98F
:102F600003E12B1C01E17ED0160EDB5016E07ED96A
:102F7000300EE66E9FD802E12B1C74E077D9DFCFCC
:102F8000E6FFB3EC21F0E552E552E552F4CF2BF029
:102F90000001F31C02E12B1C65E0050EDBCF2AF0DB
:102FA000160EDB50D8802A5409E2050EDBCFE7FF6E
:102FB000160EDB50E75E050EE7CFDBFF300EE66E48
:102FC000050ECBD94FE1390EDB2ADBCFE9FF3A0EF4
:102FD00001E3DB2ADBCFEAFF090EEFCFDBFFDB509B
:102FE0000EE044D9090EADD902E12B1C3BE0390EAD
:102FF000DB2ADBCFE9FF3A0EEDE3DB2AEBD755D82E
:1030000031E1160EDBCFE6FF080EC3D8E552E72408
:103010005DD82ED0070EDB50030A1CE0010A14E035
:10302000030A07E07BD9DBCFEEFF020EDBCFEDFF1B
:103030001FD0F5D82F6A2DAE02D02E682F682CD85D
:10304000BCD82FC0EEFF14D0EAD82DBE2E6824D8ED
:10305000B4D80ED063D9DBCFEFFF0AD07BD905E11E
:103060002B1C03E1F368F46810D0FCD801E3DB2AE1
:1030700079D9D7EF13F0010EDBCF2AF0020EDBCFA8
:103080002BF02AC0F3FF2BC0F4FF3B0EE15C02E201
:10309000E16AE552E16ECBD029D9020E3DEF19F07D
:1030A00061D90800F550DF6E1200200EE66E080EA2
:1030B000ADEF19F0B3EC21F0E552E552E552F3CF54
:1030C0002AF0F4CF2BF00001F31C12002A6E2B6AB9
:1030D000D950010F4DD92A50EE262B50ED22120067
:1030E0002E5E000E2F5AF70E2EC0DBFFF80E2FC0FB
:1030F000DBFF2EC0E9FF2FC0EAFF1200DBCFF4FF99
:10310000F350F45C1200DB50E76E040EE7CFDBFFF8
:1031100012000A0EDBCF2AF00B0EDBCF2BF00C0EC9
:10312000DBCF2CF00D0EDBCF2DF02A502B102C1006
:103130002D101200130EEECFDBFF140EEDCFDBFFD0
:10314000130EDBCF2AF0140EDBCF2BF00001800E24
:103150002B141200F70EDBCF2EF0F80EDBCF2FF082
:103160001200050EDB50E66ED950130F01D9E5525F
:10317000E750EE6EED6A12000A0EDBCF1CF00B0E6C
:10318000DBCF1DF00C0EDBCF1EF00D0EDBCF1FF0E2
:103190001200DBCFE6FF150EDBCFE6FF050EDB509E
:1031A000E552E724E552E7241200DB50CED8010EA9
:1031B000F36E060EF3CFDBFF1200EE50EFCFEAFF07
:1031C000E96E2CC0EEFF2DC0EEFF2EC0EEFF120008
:1031D000D9CFE6FFDACFE6FFE1CFD9FFE2CFDAFFC2
:1031E0001200DFCFE6FFE66A74EC22F0E552E5520A
:1031F000F3501200E76E080EE7CFDBFF1200EECFB0
:103200002AF0EECF2BF0EFCF2CF02D6A1200050E36
:10321000DBCF2AF0150EDB50D8802A541200010EA5
:10322000DBCF2CF0020EDBCF2DF02E6A1200E55220
:10323000E5CFDAFFE7CFD9FF12000A0E2AC0DBFF85
:103240000B0E2BC0DBFF1200D9500A0FB8EF19F09C
:10325000F36E070EF3CFDBFF1200EECF2AF0EFCFB5
:103260002BF01200010EDB2A020E1200FC0EDBCF47
:10327000E6FFFD0EDBCFE6FF12002A5E000E2B5AA2
:10328000F70E2AC0DBFFF80E2BC0DBFF2AC0E9FFD8
:103290002BC0EAFF1200DA20EA6EEF2AEECFF6FF2B
:1032A000000EEF22EECFF7FFEF22EECFF8FF120075
:1032B000040EDBCFE6FF130EDB50E552E75C9ADF2E
:1032C000DB5004DF060EDB501200090EDB500A0D46
:1032D000F350DF24D00FE76E090EE7CFDBFF50EF8E
:1032E00018F0DB50F36E050E7EEF18F0F70EDBCF13
:1032F0002AF0F80EDBCF2BF01200DFCFE6FF5AEFFB
:1033000018F028DF030EECDEFFEF18F0ACEC13F042
:10331000E552E552E552E55200091200BDDEEE50DD
:10332000EFCFEAFFE96E010E1200130EDB50F36ED1
:10333000040E7EEF18F0040EDB50F36E090E7EEFE4
:1033400018F0DBCFE6FF5AEF18F0E76E050EE7CF77
:10335000DBFF12008BDF7DEF19F0DBCFE6FF86DFAE
:1033600086EF19F0D950F90FE96EFF0E4BEF19F007
:0A337000E96E000EDA20EA6E12008A
:06337A00040120511F0BAD
:10338000010801E060D004012051600BE842E842EE
:10339000E842E842E842010801E055D00401245126
:1033A00004E00401240501E04ED004012151230A68
:1033B00048E0010A40E0030A30E0010A25E0240A5F
:1033C00022E0070A1FE0010A1CE0030A11E0010ADB
:1033D00001E038D00101030EC16F0101A90EC26FD7
:1033E000010EC36F0101C9930101080EC66F2BD0F6
:1033F0000101030EC16F0101A90EC46F010EC56F5B
:1034000022D021D020D01FD00101030EC16F0101B5
:10341000A10EC46F010EC56F16D00101030EC16F5E
:103420000101A10EC26F010EC36F0101C993010119
:10343000070EC66F08D00101030EC16F22C4A8F1A8
:1034400002D001D000D012000101A16BC20EA26F08
:10345000010EA36FA46B0101A56B0101A66B010115
:10346000080EA76F01019A6B0101996B1A0E726E1B
:103470001E0E736E0401000E166F050E176F040109
:10348000400E146F0401400E196F0401080E1A6FEC
:10349000050E1B6F0401880E186F0401480E1E6F85
:1034A000050E1F6F0401400E1C6F1200D9CFE6FFFE
:1034B000E1CFD9FF0101996B040118BF39D0FC0E8F
:1034C000DBCF2AF004011951D8802A5403E2FC0E04
:1034D00019C4DBFF0101996BFC0EDB500101995D02
:1034E0001CE201019951EA6A080FE96E050EEA2211
:1034F000EF50E66E01019951E76EFD0EDBCFE9FF5B
:10350000FE0EDBCFEAFFE750E926000EEA22E55285
:10351000E750EF6E0101992BDFD70401400E196FC0
:10352000400E040118170401187D880E04011813B9
:103530000101995100D0E552E7CFD9FF1200D9CF50
:10354000E6FFE1CFD9FFE65201019A5101E031D007
:10355000DF6ADF2ADF502A6E2B6A2A5002E1010E51
:103560002B1801E10BD0FD0EDBCFE9FFDB2AFE0EAD
:10357000DBCFEAFF01E3DB2AEF50EBE1DF502A6EFD
:103580002B6AD950FD0FE96EFF0EDA20EA6E2A5041
:10359000EE5E2B50ED5ADF06FD0EDBCF9BF1FE0EEB
:1035A000DBCF9CF1DFCF9FF10101A06B0101010E88
:1035B0009A6FE552E552E7CFD9FF1200D9CFE6FF67
:1035C000E1CFD9FFE65201019A5101E033D0DF6A21
:1035D000DF2ADF502A6E2B6AFF0E2A1801E12B50DA
:1035E00001E10CD0FD0EDBCFF6FFDB2AFE0EDBCFB8
:1035F000F7FF01E3DB2A0800F550EAE1DF502A6E0D
:103600002B6AD950FD0FE96EFF0EDA20EA6E2A50C0
:10361000EE5E2B50ED5ADF06FD0EDBCF9BF1FE0E6A
:10362000DBCF9CF1DFCF9FF10101010EA06F010103
:10363000010E9A6FE552E552E7CFD9FF1200D9CFBC
:10364000E6FFE1CFD9FFE65204011CBF7DD0030E97
:1036500001019A5D02E101019A6B01019A5101E1B8
:1036600073D0020E01019A5D06E104011D6B010198
:10367000030E9A6F61D001019A055EE1400E2A6E39
:103680002B6A01019F512A5C000E2B5803E2400E69
:10369000DF6E02D09FC1DFFFDFCF1DF4DF500101DD
:1036A0009F5D01019F6F0101480E9D6F050E9E6F8A
:1036B0000101A00518E1DF5015E09BC1F6FF9CC198
:1036C000F7FF0800F5509DC1E9FF9EC1EAFFEF6ECC
:1036D00001019D2B000E9E2301019B2B000E9C23BC
:1036E000DF06E9D716D0DF5014E09BC1E9FF9CC18B
:1036F000EAFFEF509DC1E9FF9EC1EAFFEF6E0101B5
:103700009D2B000E9E2301019B2B000E9C23DF06A8
:10371000EAD701019F5110E104011D512A6E2B6A65
:10372000400E2A1801E12B5004E10101020E9A6FAC
:1037300003D00101030E9A6F400E04011C1704010F
:103740001C7D880E04011C13E552E552E7CFD9FF1A
:02375000120065
:0E3752006C5002E0000E01D0010E00090BE0E9
:10376000040100513C0BE842E8420D0802E10CD88C
:1037700001D042D808D06C5002E0000E01D0010EFA
:10378000040901E04BD81200D9CFE6FFE1CFD9FF01
:10379000E6520101C06B0101C16B0101C66BC76B31
:1037A00046EC1DF0DF6ADF502A6E2B6A010E2A5CA0
:1037B000000E2B581BE20101C15101E017D0F76A3E
:1037C000DF34FE0BF736F66E2D0EF626420EF7228C
:1037D0000900F5CF2AF00800F5CF2BF004D02BC05C
:1037E000FAFF2A50F96EFBDFDF2ADDD7F0D8E55269
:1037F000E552E7CFD9FF1200020E0101C05D0CE1D6
:10380000A4D8040100BD04D00401C80E006F03D089
:103810000401880E006F01D029D91200040E0101A5
:10382000C85D0CE122C46EFF6E50000804E2010185
:10383000050EC86F03D00101030EC86F0101C0055A
:103840000CE10DD8040104BD04D00401C80E046FBE
:1038500003D00401880E046F01D008D91200D9CF1B
:10386000E6FFE1CFD9FF020EE1260101080EC65D99
:10387000000EC75905E2C6C1DEFFC7C1DDFF03D098
:10388000080EDE6EDD6A0401049304010491010E4A
:10389000DB5004010413DFCF05F4000EDB500101FF
:1038A000C65F010EDB500101C75B0101280EC46F2A
:1038B000040EC56F0101C9A320D0D9CFE9FFDACF2B
:1038C000EAFFEE50ED1018E0C2C1F6FFC3C1F7FFEA
:1038D0000800F550C4C1E9FFC5C1EAFFEF6E010160
:1038E000C42B000EC5230101C22B000EC323DF062B
:1038F000010E01E2DB06E1D71ED0D9CFE9FFDACF16
:10390000EAFFEE50ED1017E0C2C1E9FFC3C1EAFFC4
:10391000EF50C4C1E9FFC5C1EAFFEF6E0101C42B3E
:10392000000EC5230101C22B000EC323DF06010ECA
:1039300001E2DB06E2D7020EE15C02E2E16AE55257
:10394000E16EE552E7CFD9FF1200D9CFE6FFE1CF14
:10395000D9FF020EE126030E04010015E76E010EE9
:10396000E7CFDBFF01C4DFFFDE500101C627DD50DA
:103970000101C7230101280EC26F040EC36FD9CF06
:10398000E9FFDACFEAFFEE50ED1017E0C2C1E9FF20
:10399000C3C1EAFFEF50C4C1E9FFC5C1EAFFEF6E42
:1039A0000101C42B000EC5230101C22B000EC3234D
:1039B000DF06010E01E2DB06E2D7020EE15C02E265
:1039C000E16AE552E16EE552E7CFD9FF12006D984A
:1039D0000101C1510FE10401080E016F0401200E25
:1039E000026F040E036F0401840E006F0401840E45
:1039F000046F3BD0040120AF25D00101C651040162
:103A0000265D0101C7510401275904E226C4C6F10D
:103A100027C4C7F124DF0101010EC06F0401080EA5
:103A2000016F0401200E026F040E036F0401800E6B
:103A3000006F0401280E066F040E076F0401C80E04
:103A4000046F13D00101020EC06F0401056B040165
:103A5000C80E046F0401080E016F0401280E026FE6
:103A6000040E036F0401C80E006F12000101C06B49
:103A70000401080E016F0401200E026F040E036F93
:0C3A80000401880E006F0401046B1200AA
:043A8C0004012051C0
:103A9000600BE842E842E842E842E842000901E0FF
:103AA00058D004012151070A53E00B0A51E0070ADC
:103AB00042E0010A2CE00B0A28E0020A26E0030A91
:103AC00022E0080A12E0010A0EE00F0A0AE0030AE7
:103AD00001E03ED00101010EC16F0101040EC86F6B
:103AE00038D038D836D093D834D00101010EC16F08
:103AF0000101CA0EC26F010EC36F0101C99301011A
:103B0000010EC66F26D0ABD824D0F9D822D001013F
:103B1000010EC16F040124510101C26FC36BCB0EB2
:103B20000101C227010E0101C3230101C993010153
:103B3000010EC66F0ED00101010EC16F04012451A8
:103B4000EA6ACB0FE96E010EEA2222C4EFFF01D030
:103B500000D01200800E0401205D58E104012351C1
:103B6000030A34E0010A10E0030A01E04DD001012C
:103B7000010EC16F0101620EC26F410EC36F120EC2
:103B80000101C66FC76B40D00101010EC16F040176
:103B90002251F66EF76AD890F636F736230EF626DF
:103BA000420EF7220900F5CFC2F10A00F5CFC3F1AA
:103BB000020E0101F76AC225F66EC351F722090011
:103BC000F5CFC6F10A00F5CFC7F11ED00101010EF5
:103BD000C16F04012251F66EF76AD890F636F736B7
:103BE000270EF626420EF7220900F5CFC2F10A0091
:103BF000F5CFC3F1C2C1F6FFC3C1F7FF0800F5500E
:103C00000101C66FC76B00D00101C9831200010119
:103C1000010EC16F0F0EE66E710EE66E0F0EE66EB0
:103C200081EC1FF0E552E552E552010EE66ECB0E37
:103C3000E66E010EE66E81EC1FF0E552E552E552AC
:103C400022C4CAF10401225104E10101050EC86F2A
:103C500005D00101060EC86F24EC1AF01200040111
:103C6000286B0401296B040120511F0B020A14E088
:103C7000030A0EE0010A01E034D00101010EC16F18
:103C8000040128810101C9A102D00401288329D09F
:103C90000101010EC16F25D00101010EC16F0401A8
:103CA00024510F0B080DF3502B6A000F2A6E040EDF
:103CB0002B2204012451800B01E0010E040DF3506E
:103CC00001012A24C46F000E2B20C56FC4C1E9FF77
:103CD000C5C1EAFFEF50040B03E00401010E286F99
:103CE00000D00101C1050AE10101280EC26F040ED6
:103CF000C36F0101C9930101020EC66F12000401D6
:103D0000220511E1040120511F0B00090CE1010102
:103D1000010EC16F030E0401215D03E10101C981A0
:103D200002D00101C991040122513EE10401205158
:103D30001F0B020839E1040124510F0B000934E084
:103D40000101010EC16F040124510F0B080DF35046
:103D50002B6A000F2A6E040E2B2204012451800BC3
:103D600001E0010E040DF35001012A24C46F000E7E
:103D70002B20C56F030E0401215D07E1840EC4C131
:103D8000E9FFC5C1EAFFEF6E0FD0040124AF06D0F2
:103D9000C4C1E9FFC5C1EAFFEF6A06D0880EC4C1FD
:0A3DA000E9FFC5C1EAFFEF6E120053
:063DAA006DA610D802D046
:103DB0006DB614D80101C80509E16DBA07D0686A6B
:103DC000696A698069880101020EC86F12006D6A14
:103DD000696A6D860101010EC86F12006D6A696A19
:103DE0000101C86B1200FADF12000101C85101E1A4
:103DF0003AD06850040B04E06950040B01E03CD851
:103E00006DB231D06850010B04E06950010B01E044
:103E100056D86850100B04E06950100B01E024D80C
:103E20006850400B04E06950400B01E03DD86850F9
:103E3000200B04E06950200B01E038D86850020BD9
:103E400004E06950020B01E038D8030E0101C85D9F
:103E500001E209D06850080B06E06950080B03E046
:103E6000A9EC1BF068961200698468986D82A19A8B
:103E7000A08A0300A09A12006D92699468941200BF
:103E80000101C9A110D0F8DF6D840101080ED06FC7
:103E9000070ED16F0101D007000ED15B0101D05197
:103EA000D111F8E16D941200689C120070A003D04B
:103EB00036EC1DF07090689A1200689212006A6ADF
:103EC000686A9F0E6B6E7B0E696E6E6A0F0EE66EF1
:103ED000710EE66E0F0EE66E14D8E552E552E5520D
:103EE000160E706E68A602D06896FCD76D9836ECF8
:103EF0001DF00101C9910101CA6B0101030EC86FD8
:103F00001200D9CFE6FFE1CFD9FFFD0EDBCFE9FFED
:103F1000FE0EDBCFEAFFFC0EDB5004E0EE6AFC0E87
:0C3F2000DB06F9D7E552E7CFD9FF12000D
:043F2C0053746174F5
:103F300075733D25690D0A002135204572723A20BE
:103F40004E65656420636F6D6D61206E6578742CBD
:103F500020666F756E643A20272563270D0A00508E
:103F6000492C2531750D0A004D522C253033750D25
:103F70000A002C25303475004100492C2530336966
:103F80002C253033692C253033690D0A0021382067
:103F90004572723A20556E6B6E6F776E20636F6D4F
:103FA0006D616E642027256325633A2532582532DA
:103FB00058270D0A002138204572723A20556E6B41
:103FC0006E6F776E20636F6D6D616E642027256361
:103FD0003A253258270D0A002137204572723A20BF
:103FE0004578747261207061726D617465720D0A3A
:103FF000002136204572723A20496E76616C696400
:1040000020706172616D7465722076616C75650DEA
:104010000A002134204572723A204D697373696E2B
:104020006720706172616D657465722873290D0A6D
:10403000002133204572723A20525820427566663C
:104040006572206F76657272756E0D0A00213220DE
:104050004572723A20545820427566666572206F28
:1040600076657272756E0D0A002131200D0A0021ED
:0540700030200D0A00E4
:0A4076001FC029F01EC028F01DC075
:1040800027F01D502202F4CF1BF0F3CF1AF01E5080
:104090002302F4CF1DF0F3CF1CF02202F3501B26B5
:1040A000F4501C22E86A1D2227502302F3501B26DD
:1040B000F4501C22E86A1D221F502202F3501C26D5
:1040C000F4501D221F5023021E6AE86A1E22F3507C
:1040D0001D26F4501E2227502402F3501C26F450B3
:1040E0001D221F6AE86A1E221F2228502402F35054
:1040F0001D26F4501E22E86A1F2229502402F35084
:104100001E26F4501F22000C1FC029F01EC028F0EC
:104110001E502302F4CF1DF0F3CF1CF01F502402D9
:10412000F4CF1FF0F3CF1EF02302F3501D26F450FE
:104130001E22E86A1F2228502402F3501D26F45044
:104140001E22E86A1F2224AEAAEF20F028501E5E2D
:1041500029501F5A29AE000C23501E5E24501F5AAE
:02416000000C51
:0E4162001201000202000008D8040A0000004A
:10417000010200010902430002010080320904002B
:1041800000010202010005240010010424020205BE
:10419000240600010524010001070582030800022E
:1041A00009040100020A00000007050302400000A4
:1041B000070583024000000403090434034D00692D
:1041C00000630072006F00630068006900700020E7
:1041D0000054006500630068006E006F006C006FA3
:1041E0000067007900200049006E0063002E003453
:1041F000034300440043002000520053002D0032CE
:104200000033003200200045006D0075006C006135
:1042100000740069006F006E002000440065006DAE
:0F422000006F0074417441B741BB41EF417A33E5
:104230002A0EF66E080EF76E000EF86E02010900E7
:10424000F550FB6F0900F550FC6F03E1FB6701D0EF
:104250003DD00900F550F66F0900F550F76F0900E1
:10426000F550F86F09000900F550E96E0900F550A6
:10427000EA6E090009000900F550F96F0900F550D0
:10428000FA6F09000900F6CFFDF2F7CFFEF2F8CF82
:10429000FFF2F6C2F6FFF7C2F7FFF8C2F8FF02011D
:1042A000F95302E1FA5307E00900F550EE6EF90701
:1042B000F8E2FA07F9D7FDC2F6FFFEC2F7FFFFC228
:0E42C000F8FF0201FB07000EFC5BBFD71200E7
:0242CE00D9CF46
:1042D000E6FFDACFE6FFE1CFD9FFE2CFDAFFE65221
:1042E000E652E652E652D950FB0F2A6EFF0EDA2054
:1042F0002B6E2AC0DEFFDD6EDECFE6FFDDCFE6FFF0
:10430000FB0EDBCFE6FFFC0EDBCFE6FFFD0EDBCFC7
:10431000E6FFD2C1E6FFD3C1E6FFC2EC13F02A6E7E
:10432000070EE15C02E2E16AE552E16E2A50020EFC
:10433000F3CFDBFF030EF4CFDBFF020EDBCF2AF05F
:10434000030EDBCF2BF02AC0F3FF2BC0F4FF040ECB
:10435000E15C02E2E16AE552E16EE552E5CFDAFFA7
:06436000E7CFD9FF1200B7
:0A436600D9CFE6FFDACFE6FFE1CF82
:10437000D9FFE2CFDAFFFB0EDBCF2AF0FC0EDBCF5A
:104380002BF00001800E2B141AE1FB0EDBCFE9FFAE
:10439000FC0EDBCFEAFFEECFF3FFEDCFF4FFEE2A0A
:1043A000000EEF22F3CFE9FFF4CFEAFFFD0EDBCFE3
:1043B000EFFFEF502B6AF36E2BC0F4FF10D0FB0E13
:1043C000DB50FE0806E1FD0EDBCFE6FFE7EC22F056
:1043D00005D0FD0EDBCFE6FFB3EC07F0E552E5526A
:0A43E000E5CFDAFFE7CFD9FF1200A6
:0643EA001C502102F3CF7C
:1043F00018F0F4CF19F02202F3501926000EF42021
:104400001A6E1C502302F3501A26000EF4201B6E65
:104410001C502402F3501B261D502102F350192674
:10442000F4501A22000E1B221D502202F3501A26AD
:10443000F4501B221D502302F3501B261E50210254
:10444000F3501A26F4501B221E502202F3501B2652
:0A4450001F502102F3501B2612003A
:06445A00FE0EE3CFE9FFB6
:10446000FF0EE3CFEAFFF36AF46AEE5203E0F34A89
:10447000F42AFBD71200FF0EE3CFF8FFE552FF0E40
:10448000E3CFF7FFE552FF0EE3CFF6FFE552E66A12
:10449000E66AE66A0900F55209E0FD0EE32A05E145
:1044A000FE0EE32A02E1FF0EE32AF4D7FD0EE3CF6E
:1044B0001DF0FE0EE3CF1EF0FF0EE3CF1FF0120043
:1044C000FF0EE124E96EFF0EE220EA6EEDCFF4FF6D
:1044D000EFCFF3FFF46607D0600EF36404D07B0ED9
:1044E000F36001D0F39A1200F36AF46AFF0EE1243C
:1044F000E96EFF0EE220EA6EED6607D02F0EEF6444
:0C45000004D03A0EEF6001D0F32A120044
:04450C001B6A1A6AA2
:10451000196A186A200EE76ED8901C361D361E36B2
:104520001F36183619361A361B362150185C2250A1
:10453000195823501A5824501B5809E32150185E6B
:104540002250195A23501A5A24501B5A1C2AE72E5B
:04455000E4D712009A
:0C45540005D811D88FEC06F0FCD712003F
:104560000F0EC112140E6F6E0101C86B0101C96BF1
:104570000101CA6BC4EC05F01200D5EC1EF06FBE51
:0C45800002D0F5EC1EF01FEC1BF0120046
:04458C004F4B0D0A7A
:10459000000D0A00554257204657204420566572A8
:0D45A00073696F6E20312E342E350D0A0028
:0245AE00000EFD
:1045B000F36E00EE00F0040E01D81200EA6002D0A3
:0E45C000EE6AFCD7F350E9601200EE6AFCD7F9
:0245CE00FF0EDE
:1045D000E350ACBA04D0AF6AAB8EAC8A949CACA268
:0A45E000FED7AD6EF36EF46A120010
:0645EA0013EE00F023EEC9
:1045F00000F0F86A179C18EC21F0AAEC22F0FDD725
:024600001200A6
:0E460200FF0EE350E84E1200000000D000D082
:0846100000D0E82EFAD71200D9
:084618003031323334353637FE
:09462000383961626364656600CB
:04462900000000008D
:02462D00FEFF8E
:00000001FF
